:020000040000FA
:040000006D303A28FD
:08000800A000030EA100831209
:1000100005191028831601178312B23081002B288E
:1000200083160113831203140B190310A80DA90DD5
:10003000AA0DAB0DAC0DAC16FF302C02031D2B2806
:10004000FA302B02031D2B2831152A08AF0029088E
:10005000AE002808AD008B100B11210E8300A00EFE
:04006000200E090065
:0C007400203084008001840A6030040207
:10008000031C3C281230B0009F2183160C308505DC
:1000900087018312850187010730990000309A009B
:1000A000103083168E008312603083168F00831207
:1000B0000030831691008312C830831681008312AA
:1000C00031309000003083168C00831210308B008A
:1000D000831600309B001C141A088312BC00851D77
:1000E000E321831610309B001C141A088312BD00F4
:1000F000DB2181018E018F010B118B100B108C0104
:100100008B17902031199320B30B8E28031085197B
:100110000314B90DF030390203191821082281287F
:1001200064003210080031110130B7008B13203009
:10013000370783169B001C141A088312A400103082
:10014000370783169B001C141A088312A300A6000D
:100150000230A6060030370783169B001C141A08CD
:100160008312A200A7000130A7068B17321CBE28FD
:1001700022090339A200A309A409A50924082F0212
:10018000031D122923082E02031D122922082D0205
:10019000031D122901303702031DD3283D18D3282F
:1001A0003D143E14AA2102303702031DDC28BD187D
:1001B000DC28BD143E14AC2103303702031DE528B2
:1001C0003D19E5283D153E14AE2104303702031DCC
:1001D000EE28BD19EE28BD153E14B02105303702BA
:1001E000031DF7283D1AF7283D163E14B2210630AC
:1001F0003702031D0029BD1A0029BD163E14B42183
:1002000007303702031D09293D1B09293D173E14FC
:10021000B62108303702031D1229BD1B1229BD1754
:100220003E14B821B70A093037020318080096288F
:100230000130B600B300B400B500B70085018701F6
:10024000B1139020B30B5029031085190314B90D75
:10025000F030390203197729B40B502901303702E5
:100260000319C321023037020319C62103303702B4
:100270000319C921043037020319CC210530370294
:100280000319CF21063037020319D2210730370274
:100290000319D521083037020319D8219630B4004C
:1002A000311D21293111321C5A292D090339AD0084
:1002B000AE09AF092F1C21298E018F010C1C2129A9
:1002C0000C102E1E21298B1320303707BB002F085E
:1002D000BA008A2110303707BB002E08BA008A21E5
:1002E00000303707BB002D08BA008A218B17850123
:1002F0008701B70AB60109303702031C2129DB2127
:1003000008003E1C08003E101030BB003D08BA003B
:100310008A2108008B133A0883161C159A00831251
:100320003B0883169B0055309D00AA309D009C140D
:1003300064009C1898291C1183128B170800FF3049
:10034000D000D415D515D615D715D915DA15DB1566
:10035000DC150800F130BB29F230BB29F430BB2991
:10036000F830BB291F30BF292F30BF294F30BF299C
:100370008F30BF290800BD050F30D2040800BD052D
:10038000F030D204080010308506080020308506C1
:100390000800213085060800223085060800183044
:1003A0008706080021308706080009308706080004
:1003B0002930870608003D08D200031D08001130CF
:1003C000BD00D2000800B601B301B4013C1CEB290A
:1003D000BC01BC14ED29BC013C143C08B60064000F
:1003E000F129F229F329F429F529B41B0516B41FC4
:1003F0000512B30BEF29B40BEF290310B60CB608A6
:10040000031DEF290030BB003C08BA008A21080018
:100410008F08031908008F01D00F222BD00A0E304D
:100420005205031D222A541D182AD4015416302ABD
:10043000D41D1D2AD4015416302A541E302AD4014A
:10044000D414302AD41C272AD4015415302A541D20
:100450002C2AD401D415302A541E302AD401541524
:1004600001305205031D432A551D392AD501551661
:10047000512AD51D3E2AD5015516512A551E512AFD
:10048000D501D514512AD51C482AD5015515512A14
:10049000551D4D2AD501D515512A551E512AD50174
:1004A00055150B305205031D642A561D5A2AD601D4
:1004B0005616722AD61D5F2AD6015616722A561E65
:1004C000722AD601D614722AD61C692AD60156156C
:1004D000722A561D6E2AD601D615722A561E722A07
:1004E000D601561507305205031D852A571D7B2A54
:1004F000D7015716932AD71D802AD7015716932A5A
:10050000571E932AD701D714932AD71C8A2AD701BA
:100510005715932A571D8F2AD701D715932A571E8F
:10052000932AD70157151030BC1811305205031DFE
:10053000A82A591D9E2AD9015916B62AD91DA32ABF
:10054000D9015916B62A591EB62AD901D914B62A84
:10055000D91CAD2AD9015915B62A591DB22AD9017B
:10056000D915B62A591EB62AD90159155030BC18CA
:1005700051305205031DCB2A5A1DC12ADA015A16E1
:10058000D92ADA1DC62ADA015A16D92A5A1ED92AB8
:10059000DA01DA14D92ADA1CD02ADA015A15D92A52
:1005A0005A1DD52ADA01DA15D92A5A1ED92ADA01B2
:1005B0005A15E030BC18E1305205031DEE2A5B1DD0
:1005C000E42ADB015B16FC2ADB1DE92ADB015B1652
:1005D000FC2A5B1EFC2ADB01DB14FC2ADB1CF32A51
:1005E000DB015B15FC2A5B1DF82ADB01DB15FC2A0D
:1005F0005B1EFC2ADB015B152030BC182130520544
:10060000031D112B5C1D072BDC015C161F2BDC1D51
:100610000C2BDC015C161F2B5C1E1F2BDC01DC1479
:100620001F2BDC1C162BDC015C151F2B5C1D1B2BF0
:10063000DC01DC151F2B5C1E1F2BDC015C158121EE
:100640003D08D2005008D1000C305405031D05129E
:100650000C305505031D85120C305605031D051081
:100660000C305705031D85100C305905031D07106C
:100670000C305A05031D87120C305B05031D071251
:100680000C305C05031D871151080E0203186C2BFA
:1006900012305405031D051612305505031D85162D
:1006A00012305605031D051412305705031D85141D
:1006B00012305905031D071412305A05031D871601
:1006C00012305B05031D071612305C05031D8715EC
:1006D000FF305002031908008F08031D0800902006
:1006E00051080E02031C6C2B18305405031D051213
:1006F00006305405031D051618305505031D8512D7
:1007000006305505031D851618305605031D0510C6
:1007100006305605031D051418305705031D8510B6
:1007200006305705031D851418305905031D0710A1
:1007300006305905031D071418305A05031D87128A
:1007400006305A05031D871618305B05031D071276
:1007500006305B05031D071618305C05031D871165
:0A07600006305C05031D8715080034
:084000000400030002000600A9
:02400E00CC33B1
:10420000010078007A007C007E007B0079007F004E
:104210007D007A0078007E007C00FF00FF00FF0038
:104220000000F200F600FA00FE00F200F600FA00CC
:10423000FE00F200F600FA00FE00FF00FF00FF00A3
:10424000010005000500050005000900090009003E
:1042500009000D000D000D000D00FF00FF00FF0024
:10426000FF00FF00FF00FF00FF00FF00FF00FF0056
:10427000FF00FF00FF00FF00FF00FF00FF00FF0046
:10428000FF00FF00FF00FF00FF00FF00FF00FF0036
:10429000FF00FF00FF00FF00FF00FF00FF00FF0026
:1042A000FF00FF00FF00FF00FF00FF00FF00FF0016
:1042B000FF00FF00FF00FF00FF00FF00FF00FF0006
:1042C000FF00FF00FF00FF00FF00FF00FF00FF00F6
:1042D000FF00FF00FF00FF00FF00FF00FF00FF00E6
:1042E000FF00FF00FF00FF00FF00FF00FF00FF00D6
:1042F000FF00FF00FF00FF00FF00FF00FF00DD00E8
:00000001FF
